:10800000FEDF07EA000000000000000000000000A2
:108010000000000000000000000000000000000060
:108020000000000000000000000000000000000050
:108030000000000000000000000000000000000040
:108040000000000000000000000000000000000030
:02000004001FDB
:020000040020DA
:1000000002D3A0E3CD0000EBFEFFFFEA001080E585
:100010001EFF2FE1B010C0E11EFF2FE10010C0E570
:100020001EFF2FE1000090E51EFF2FE10E00A0E172
:100030001EFF2FE100C0A0E33ACF07EE4FF07FF59F
:1000400000C0A0E315CF07EE00C0A0E3D5CF07EEB8
:100050004FF07FF56FF07FF510FF2FE11EFF2FE1CE
:1000600000000FE11EFF2FE1100F11EE1EFF2FE128
:1000700010402DE908009FE5E9FFFFEB1040BDE8C7
:100080001EFF2FE15450213F10402DE91C009FE539
:10009000E3FFFFEB010010E3FBFFFF0A10009FE509
:1000A000DFFFFFEB1040BDE8FF0000E21EFF2FE185
:1000B0005450213F4050213F10402DE90C009FE556
:1000C000D7FFFFEB1040BDE8010000E21EFF2FE16B
:1000D0005450213F10402DE90040A0E11C009FE555
:1000E000CFFFFFEB200010E3FBFFFF0A0410A0E1AD
:1000F0000C009FE5C4FFFFEB1040BDE81EFF2FE1A1
:100100005450213F4050213F10402DE910009FE501
:10011000C3FFFFEB010C10E3FBFFFF1A1040BDE82B
:100120001EFF2FE15450213F70402DE90050A0E107
:100130002040A0E3044044E23504A0E10F0000E2C7
:10014000090050E33700808230008092E0FFFFEB2F
:10015000000054E3F6FFFF1A2000A0E37040BDE862
:10016000DBFFFFEA10402DE9EEFFFFEB0D00A0E3FF
:10017000D7FFFFEB0A00A0E31040BDE8D4FFFFEA81
:1001800010402DE90110A0E3D4009FE59EFFFFEB96
:100190000010A0E3CC009FE59BFFFFEB0010A0E365
:1001A000C4009FE598FFFFEB0310A0E3BC009FE5B0
:1001B00095FFFFEB0010A0E3B4009FE592FFFFEB7B
:1001C0000010A0E39C009FE58FFFFFEBC610A0E3AB
:1001D000A0009FE58CFFFFEB9C109FE59C009FE536
:1001E00089FFFFEB98009FE58DFFFFEB3F1AC0E30F
:1001F000121A81E388009FE583FFFFEB0010A0E364
:1002000080009FE580FFFFEB0040A0E30400A0E139
:10021000014084E290FFFFEB960054E3FAFFFF1ADF
:100220000319A0E360009FE577FFFFEB0040A0E328
:100230000400A0E1014084E287FFFFEB960054E355
:10024000FAFFFF1A0010A0E33C009FE56EFFFFEBF2
:100250000310A0E310009FE56BFFFFEB1040BDE82B
:100260001EFF2FE10450213F4450213F6050213FA9
:100270004C50213F5050213F4850213F0E0100007B
:100280006850213F0400203F9400203F9800203F09
:1002900010402DE91C409FE5F918A0E30400A0E1FF
:1002A00059FFFFEB0400A0E10C109FE556FFFFEBA8
:1002B0001040BDE81EFF2FE108B4003F0002F90026
:1002C00010402DE908009FE555FFFFEB1040BDE809
:1002D0001EFF2FE120B4003F70402DE954409FE500
:1002E0000400A0E14EFFFFEB4C509FE50E16C0E36B
:1002F000021681E30400A0E143FFFFEB0500A0E14B
:1003000047FFFFEB0E19C0E31C4084E20500A0E1AB
:10031000021981E33CFFFFEB0400A0E10219A0E316
:1003200039FFFFEB0400A0E10810A0E336FFFFEB6C
:100330007040BDE81EFF2FE11000203F0C00203F61
:10034000F0472DE90070A0E3E2FFFFEB8BFFFFEB2E
:100350006C029FE582FFFFEB33FFFFEB80FFFFEBBB
:100360003EFFFFEB7EFFFFEB3EFFFFEB7CFFFFEB73
:100370004900A0E356FFFFEB4800A0E354FFFFEB6A
:100380004500A0E352FFFFEB5800A0E350FFFFEB56
:100390000D00A0E34EFFFFEB0A00A0E30790A0E1F1
:1003A0000760A0E10750A0E10780A0E10740A0E1BD
:1003B00047FFFFEB33FFFFEB3A0050E32B00000A4F
:1003C0000A0050E30D00501301A0A00300A0A013E9
:1003D0002900000A2030C0E3470053E35000000A20
:1003E000013044E2140053E303F19F97F0FFFFEA6A
:1003F00060042000600420000005200000052000AB
:100400000005200000052000E0042000A8042000D2
:10041000840420008404200084042000840420003C
:1004200078042000440420004404200044042000F8
:10043000440420004404200044042000440420001C
:1004400044042000390050E3070040820992A0E1F3
:100450000F0000E2150054E3099080E14C00000A0F
:1004600008FFFFEB3A0050E3014084E2D3FFFF1A9C
:100470000140A0E3CEFFFFEA0662A0E10040A0E356
:10048000CBFFFFEA390050E3070040820662A0E19B
:100490000F0000E2066080E10668A0E12668A0E1A6
:1004A000014084E2C2FFFFEA390050E307004082C6
:1004B0000552A0E10F0000E2055080E1FF5005E287
:1004C000010055E32700000A0E40A033B8FFFF3AB1
:1004D000020055E30940A0030040A013B4FFFFEA67
:1004E000390050E3070040820552A0E10F0000E20E
:1004F000055080E1FF5005E20840A0E3ACFFFFEAB1
:10050000390050E3070040820882A0E10F0000E2BA
:10051000088080E10888A0E1288886E1014084E223
:10052000A3FFFFEA0D00A0E3E9FEFFEB2D00A0E32F
:10053000E7FEFFEB2D00A0E3E5FEFFEB0D00A0E3DF
:10054000E3FEFFEB0A00A0E3E1FEFFEB0A00A0E3FD
:10055000DFFEFFEB0209A0E3B5FEFFEB0A00A0E11E
:10056000F047BDE81EFF2FE11440A0E30700A0E123
:10057000FBFEFFEB014054E2FBFFFF1A0470A0E119
:100580000490A0E10460A0E10450A0E10480A0E197
:1005900087FFFFEA693829E02334A0E1FF3CC3E389
:1005A000699423E00800A0E1077088E00910A0E149
:1005B00095FEFFEB077089E0048088E20E40A0E31F
:0805C0007BFFFFEA78563412BC
:040000030000800079
:00000001FF
